:1000000088315B2F0000FB0000307A078A007B08F4
:100010000C3E03188A0A8200003400340034003495
:100020000034003400345F340034003400340334CE
:1000300000340334003414343E3414343E34143465
:1000400024342A347F342A34123443343334083489
:1000500066346134363449345534223450340034F3
:10006000053403340034003400341C342234413469
:1000700000340034413422341C3400341434083445
:100080003E3408341434083408343E340834083418
:100090000034503430340034003408340834083428
:1000A00008340834003460346034003400342034C0
:1000B00010340834043402343E3451344934453465
:1000C0003E34043402347F3400340034423461342A
:1000D0005134493446342234413449344934363475
:1000E0001834143412347F341034273445344534F2
:1000F000453439343E344934493449343234013496
:1001000001347134093407343634493449344934BC
:10011000363426344934493449343E340034363494
:10012000363400340034003456343634003400346D
:100130000834143422344134003414341434143464
:100140001434143400344134223414340834023466
:1001500001345134093406343E3441345934553471
:100160005E347E340934093409347E347F344934B2
:100170004934493436343E344134413441342234F4
:100180007F344134413441343E347F34493449343E
:10019000493441347F3409340934093401343E345C
:1001A0004134413449343A347F3408340834083413
:1001B0007F34003441347F344134003430344034AF
:1001C000403440343F347F340834143422344134D2
:1001D0007F3440344034403440347F3402340C3473
:1001E00002347F347F340234043408347F343E34A4
:1001F0004134413441343E347F34093409340934C4
:1002000006341E342134213421345E347F340934E1
:100210000934093476342634493449344934323483
:10022000013401347F34013401343F3440344034EC
:1002300040343F341F342034403420341F347F3462
:100240002034103420347F34413422341C3422349E
:10025000413407340834703408340734613451347D
:1002600049344534433400347F344134003400345D
:10027000023404340834103420340034003441345F
:100280007F34003404340234013402340434403402
:1002900040344034403440340034013402340434B7
:1002A0000034203454345434543478347F34443457
:1002B0004434443438343834443444344434443496
:1002C00038344434443444347F343834543454342B
:1002D00054341834043404347E340534053408347A
:1002E0005434543454343C347F34083404340434A7
:1002F0007834003444347D34403400342034403485
:1003000044343D3400347F341034283444340034D1
:10031000003441347F34403400347C340434783445
:10032000043478347C340834043404347834383475
:1003300044344434443438347C3414341434143461
:10034000083408341434143414347C3400347C34C9
:100350000834043404344834543454345434203489
:10036000043404343F34443444343C344034403462
:1003700020347C341C342034403420341C343C344D
:100380004034303440343C3444342834103428343D
:1003900044340C345034503450343C344434643499
:1003A00054344C3444340034083436344134413409
:1003B000003400347F340034003441344134363466
:1003C0000834003402340134023404340234C337B4
:1003D0006E37E531F4346F37A03AEE3474102532BD
:1003E0000000D32BA02052294127C7223A00CE2754
:1003F000D22641260001D32B412820100000C3370C
:100400006E37E531F4346F372033E134EC3AF232B1
:100410002010000120276F10F33467376136201059
:10042000201020102010201000014936EC32E73057
:100430006C10E430F43020336F39ED30741000016B
:10044000D32B492A4324A02052294127C722CD2259
:100450004E2A00015527492A25323A00CE27D226B6
:1004600041260001D32B412820100001D02A53241B
:10047000A029D71AA022D82454004937F43267178C
:10048000A02AEE347410CD34EE340001CF25492972
:10049000C1255510C12AC4244F0032183218AD2688
:1004A000E13C2D1936102000203085006D3084008D
:1004B00000080319682A0A30F800F701F70B5E2AD2
:1004C000F80B5D2A5F30F700F70B642A800B5B2A7C
:1004D0000800FF3021008C008D0024008D002100D9
:1004E000951322008C1021008C1422000C10210086
:1004F0000C1422008C1321008C1722000C132100F5
:100500000C170C1122000C1521008C1588312000CD
:10051000852F2100B60123009101951315141308AE
:100520004F3C0319962A2100B60A2300013091009E
:100530009513151413084B3C0319A12A2100B60A80
:10054000230002309100951315141308493C031938
:10055000AC2A2100B60A230003309100951315142C
:100560001308523C0319B72A2100B60A23000430AD
:100570009100951315141308413C0319C22A210058
:10058000B60A2300053091009513151413084B3C4F
:100590000319CD2A2100B60A2300063091009513D5
:1005A00015141308553C0319D82A2100B60A230054
:1005B00021003608F800883120008F2F2300910198
:1005C0004F309300951315150B08F7008B1355301A
:1005D0009600AA30960095149518EC2A1511770804
:1005E0008B04013091004B309300951315150B08C7
:1005F000F7008B1355309600AA3096009514951885
:10060000FF2A151177088B040230910049309300BE
:10061000951315150B08F7008B1355309600AA306B
:10062000960095149518122B151177088B0403303A
:10063000910052309300951315150B08F7008B139A
:1006400055309600AA30960095149518252B151153
:1006500077088B04043091004130930095131515F1
:100660000B08F7008B1355309600AA3096009514AE
:100670009518382B151177088B04053091004B30F5
:100680009300951315150B08F7008B135530960042
:10069000AA309600951495184B2B151177088B04EA
:1006A0000630910055309300951315150B08F7008F
:1006B0008B1355309600AA309600951495185E2B32
:1006C000151177088B042000A1010A302300910046
:1006D0002000210823009300951315150B08F7003F
:1006E0008B1355309600AA30960095149518762BEA
:1006F000151177088B042000A2010B302300910014
:100700002000220823009300951315150B08F7000D
:100710008B1355309600AA309600951495188E2BA1
:10072000151177088B042000A3010C3023009100E1
:100730002000230823009300951315150B08F700DC
:100740008B1355309600AA30960095149518A62B59
:10075000151177088B042000A4010D3023009100AF
:100760002000240823009300951315150B08F700AB
:100770008B1355309600AA30960095149518BE2B11
:10078000151177088B042000A50114302300910077
:100790002000250823009300951315150B08F7007A
:1007A0008B1355309600AA30960095149518D62BC9
:1007B000151177088B0488312000952F0A3023000B
:1007C00091009513151413082000A1000B3023008D
:1007D00091009513151413082000A2000C3023007B
:1007E00091009513151413082000A3000D30230069
:1007F00091009513151413082000A4001430230051
:1008000091009513151413082000A5008831982F26
:1008100022000C150230F700F70B0C2C00008C1195
:1008200021008C1122000C112000080021008C15E1
:1008300022000C150C112000080022008C11210050
:100840008C1122000C150C112000080022008C11C4
:1008500021008C110230F700F70B2C2C0000220035
:100860000C1521008C15200008002100CC1F3C2C09
:10087000200016243E2C210020001D2421004C1FA6
:10088000452C20001624472C210020001D24210087
:10089000CC1E4E2C20001624502C210020001D249C
:1008A00021004C1E572C20001624592C210020001A
:1008B0001D242100CC1D602C20001624622C210058
:1008C00020001D2421004C1D692C200016246B2CB7
:1008D000210020001D242100CC1C722C2000162495
:1008E000742C210020001D2421004C1C7B2C200096
:1008F00016247D2C210020001D242100CE018C1502
:1009000022000C1520008C19832C22000C118C1154
:1009100021008C114E08643C031D922C0130F8001C
:10092000952C952C0030F800952CF80803199E2C76
:10093000200026240130F8009D2C21002000080012
:10094000200BC62C082478302100CC002000352450
:100950002100CC0120003524AD302100CC00200046
:1009600035248B302100CC0020003524AF3021000D
:10097000CC0020003524A1302100CC0020003524FB
:10098000C8302100CC00200035242624A008031DF7
:10099000ED2C082478302100CC00200035242100E3
:1009A000CC01200035248D302100CC0020003524DE
:1009B00014302100CC0020003524AF302100CC00C1
:1009C00020003524A1302100CC0020003524C8307F
:1009D0002100CC002000352426248831A12F200BB3
:1009E000362D2100B8013808073C031C352D2000A6
:1009F000082478302100CC00200035242100CC01CF
:100A0000200035242100CC012000352410302100A5
:100A1000CC002000352421003808B038B900CC00C3
:100A2000200035242624082478302100CC00200022
:100A3000352440302100CC00200035242100B701AE
:100A4000B601B708031D302D3608833C031C302D3A
:100A5000CC01200035242100B60A0319B70A212D44
:100A6000200026242100B80AF32C2000A008031D32
:100A7000852D082478302100CC0020003524210069
:100A8000CC012000352420302100CC00200035246A
:100A90002100CC012000352421302100CC00200091
:100AA00035242100CC01200035247F302100CC00EA
:100AB0002000352422302100CC00200035242100E4
:100AC000CC012000352407302100CC002000352443
:100AD0002624082478302100CC0020003524403022
:100AE0002100CC00200035242100B701B6013708D1
:100AF000033C031C832DCC01200035242100B60AC1
:100B00000319B70A772D20002624080021003E088B
:100B10002000A60021003F082000A7000800F701E0
:100B2000F80121004B0803104C18F707F70CF80CDC
:100B3000CC18F707F70CF80C4C19F707F70CF80C62
:100B4000CC19F707F70CF80C4C1AF707F70CF80C50
:100B5000CC1AF707F70CF80C4C1BF707F70CF80C3E
:100B6000CC1BF707F70CF80C200008002100450803
:100B70001F3C03184D2E200028082602031DC42DFB
:100B8000290827020319022E082478302100CC00FE
:100B9000200035242100CC01200035242708A9009D
:100BA000B0382100CB00CC0020003524200BE52DEF
:100BB00026082100CB000630CC0020008F25023013
:100BC00078072100C600EF2D200026082100CB0069
:100BD0000630CC0020008F2578082100C60046088A
:100BE0000F39CB00CC00200035242100460EF70041
:100BF0000F30F70577080F391038CB00CC002000F4
:100C000035242624082478302100CC002000352407
:100C100040302100CC002000352420302100450246
:100C2000C800CA014A08043C031C452ECC014808F0
:100C3000CB00CE010530CD001030CF00F701FA0116
:100C4000CC0CCB0C031C2A2E4D08F7070318FA0A0C
:100C50004E08FA07FA0CF70CF90CF80CCF0B202E03
:100C60007908CC007808CB004A084B07F800003020
:100C70004C3DFA007808200003202100CB00CC0076
:100C8000200035242100CA0A122ECC012000352470
:100C900026242608A60AA800210020000800230018
:100CA000951715140000000013087F390319912EC1
:100CB0002100BE00230011082100BF0023001208FC
:100CC0002100C0003E08C5002000B62521003F08D5
:100CD000230091002100400823009200951715146D
:100CE00000000000130D140D7F390319912E21000F
:100CF000BE00230011082100BF00230012082100BC
:100D0000C0003E08C5002000B62521003F08230092
:100D100091002100400823009200910A0319920AD1
:100D2000502E200008002300951715140000000025
:100D30000318BE2E13087F392100C00023001108BC
:100D40002100C100230012082100C2004008C50094
:100D50002000B6252100410823009100210042080F
:100D60002300920095171514000000002100BF0B0E
:100D7000BA2EBC2E2300BE2EE12E2300130D140D1F
:100D80007F392100C000230011082100C100230089
:100D900012082100C2004008C5002000B62521002D
:100DA0004108230091002100420823009200910A8B
:100DB0000319920A03102100BF0BDF2EE12E200041
:100DC000932E2000080021004608F8014502031870
:100DD000EC2E4508F700F82EF7010830C700C50DC6
:100DE000F70D460877020318F700F80DC70BEF2E32
:100DF0002000080020302100401E3030C1003F0894
:100E0000F700BF1F0A2FF709F70A7708BF002D3038
:100E1000C100C0173F08C5006430C6002000E326AB
:100E200077082100BF0030307807C2003F08C500B6
:100E30000A30C6002000E326303077072100C400C6
:100E400030307807C3004108F700C01D292FC01FAC
:100E50004011401A362FC01F512F4019512F7708CB
:100E6000C200C018512F7708C300512F3030420202
:100E7000031D512F7708C2002030C100C01D442F30
:100E80004011C014C01FC01030304302031D512F49
:100E90007708C3002030C200C01D442FC010C01FFF
:100EA0004010401D582F4108C5002000B6252100E4
:100EB000C01C5F2F4208C5002000B6252100401C41
:100EC000662F4308C5002000B62521004408C50050
:100ED0002000B62508002100B20120000D1C732F50
:100EE0002100B20A20002100B30120008D1C7B2FBD
:100EF0002100B30A20002100B40120000D1D832F22
:100F00002100B40A20002100B50120008D1D8A2F88
:100F10002100B50A200008002100BE010630BF00F4
:100F200020008625013021003D07BE00E730230068
:100F3000910001309200031010302100BF0020000A
:100F4000932621003E08BF001F30C0002000FA2673
:100F50002100BE010730BF0020008625F1302300AC
:100F600091000130920020004F26013021003D0702
:100F70008400203085000318850A8008031DC92FCE
:100F8000F730230091000130920020004F26D02F2F
:100F90002100FB30230091000130920020004F26F9
:020FA000080047
:101000002100BE01BF0180312000862588312030BB
:101010002300910002309200803120004F26883159
:101020000D1A202802302100B700FA30BD008031AF
:101030002000542288312100B70B152820001028E9
:101040000D1EE9282100B6013608033C031C752853
:1010500001303607B700BE013708BF0080312000DD
:1010600086258831013021003607B7002A30230059
:10107000910002309200031004302100BF00803143
:1010800020009326883121003708BF001F30C000A0
:1010900080312000FA2688313A302100C5008031A5
:1010A0002000B62588310130210036078400203029
:1010B00085000318850A8008031D69282E30230047
:1010C000910002309200803120004F268831722832
:1010D0002100323023009100023092008031200044
:1010E0004F2688312100B60A2428BE010630BF00F1
:1010F000803120008625883136302300910002306F
:101100009200803120004F26883180316B27883152
:101110002100B6013608033C031CE728623036077D
:101120008400203085000318850A8008031DE52807
:10113000013036078400203085000318850A800AB4
:10114000013036078400203085000318850A000826
:10115000013980000A303607B700013036078400B5
:10116000203085000318850A0008B80037082300DE
:1011700091002100380823009300951315150B08E2
:10118000F7008B1355309600AA30960095149518E9
:10119000C728151177088B046230210036078400B8
:1011A000203085000318850A8008031DDE28803161
:1011B00020006B2788312300CC2821000A30BD0095
:1011C00080312000542288312100B60A8A2820006C
:1011D00020288831EA2F01302100BC00B601BA0076
:1011E000BB00FB00F600F500F4000C1220002508FF
:1011F0002100BD00803120008C278831643021001F
:10120000BD0080312000542288312100BB08031921
:10121000582F20000D180E29F00110290130F00080
:101220008D181429F10116290130F1000D191A2920
:10123000F2011C290130F2008D192029F301222925
:101240000130F300013025078400203085000318A9
:10125000850A800803193A2970082100B90071082D
:10126000F0003908F1007208B9007308F20039087B
:10127000F30020003230FE002100AD01AC01C93086
:10128000AB000E30AA0022000C1220002508031922
:101290005329013A0319942A033A0319D52B013A29
:1012A0000319162D582E8C1C6E292100AA08031D27
:1012B0006429AB08031D6429AC08031D6429AD082B
:1012C000031D642920006E29FF30AA07031CAB0709
:1012D000031CAC07031CAD07200053291F30F70087
:1012E000F70B702973290F30F700F70B7529782950
:1012F0008C1C7C29FC177D29FC131F30F700F70B91
:101300007F2982298C1C86297C1787297C131F3012
:10131000F700F70B89298C298C1C9029FC16912940
:10132000FC121F30F700F70B932996298C1C9A2981
:101330007C169B297C121F30F700F70B9D29A029F2
:101340008C1CA429FC15A529FC111F30F700F70BF4
:10135000A729AA298C1CAE297C15AF297C111F3026
:10136000F700F70BB129B4298C1CB829FC14B92952
:10137000FC101F30F700F70BBB29BE298C1CC229BB
:101380007C14C3297C101F30F700F70BC529C8292E
:101390008C1CCF29FE080319CF29FE03C8291F3052
:1013A000F700F70BD129D4290F30F700F70BD62916
:1013B000D9298C1CDD29FD17DE29FD131F30F7000C
:1013C000F70BE029E3298C1CE7297D17E8297D1319
:1013D0001F30F700F70BEA29ED298C1CF129FD16C7
:1013E000F229FD121F30F700F70BF429F7298C1CA6
:1013F000FB297D16FC297D121F30F700F70BFE2913
:10140000012A8C1C052AFD15062AFD111F30F70044
:10141000F70B082A0B2A8C1C0F2A7D15102A7D1128
:101420001F30F700F70B122A152A8C1C192AFD14FD
:101430001A2AFD101F30F700F70B1C2A1F2A8C1CDC
:10144000232A7D14242A7D101F30F700F70B262A4B
:10145000292A0F30F700F70B2B2A2E2A21008C1097
:101460001F30F700F70B322A352AF00803193A2A01
:101470008C143B2A8C101F30F700F70B3D2A402AB2
:10148000F1080319452A8C14462A8C101F30F700E6
:10149000F70B482A4B2AF2080319502A8C14512AB8
:1014A0008C101F30F700F70B532A562AF308031944
:1014B0005B2A8C145C2A8C101F30F700F70B5E2A15
:1014C000612AF4080319662A8C14672A8C101F30CD
:1014D000F700F70B692A6C2AF5080319712A8C1496
:1014E000722A8C101F30F700F70B742A772AF6083F
:1014F00003197C2A8C147D2A8C101F30F700F70BFF
:101500007F2A822AFB080319872A8C14882A8C10C8
:101510001F30F700F70B8A2A8D2A8C141F30F70032
:10152000F70B902A932A5A2E0C1CAF2A2100AA08E6
:10153000031DA52AAB08031DA52AAC08031DA52A77
:10154000AD08031DA52A2000AF2AFF30AA07031CFF
:10155000AB07031CAC07031CAD072000942A1F3007
:10156000F700F70BB12AB42A0F30F700F70BB62AB1
:10157000B92A0C1CBD2AFC17BE2AFC131F30F70029
:10158000F70BC02AC32A0C1CC72A7C17C82A7C1355
:101590001F30F700F70BCA2ACD2A0C1CD12AFC16E3
:1015A000D22AFC121F30F700F70BD42AD72A0C1CC2
:1015B000DB2A7C16DC2A7C121F30F700F70BDE2AB0
:1015C000E12A0C1CE52AFC15E62AFC111F30F70065
:1015D000F70BE82AEB2A0C1CEF2A7C15F02A7C1169
:1015E0001F30F700F70BF22AF52A0C1CF92AFC141D
:1015F000FA2AFC101F30F700F70BFC2AFF2A0C1CFC
:10160000032B7C14042B7C101F30F700F70B062BE8
:10161000092B0C1C102BFE080319102BFE03092BA1
:101620001F30F700F70B122B152B0F30F700F70BBD
:10163000172B1A2B0C1C1E2BFD171F2BFD131F30F5
:10164000F700F70B212B242B0C1C282B7D17292BA3
:101650007D131F30F700F70B2B2B2E2B0C1C322B7E
:10166000FD16332BFD121F30F700F70B352B382BEF
:101670000C1C3C2B7D163D2B7D121F30F700F70B09
:101680003F2B422B0C1C462BFD15472BFD111F3009
:10169000F700F70B492B4C2B0C1C502B7D15512BB5
:1016A0007D111F30F700F70B532B562B0C1C5A2BB8
:1016B000FD145B2BFD101F30F700F70B5D2B602B2B
:1016C0000C1C642B7D14652B7D101F30F700F70B6D
:1016D000672B6A2B0F30F700F70B6C2B6F2B210059
:1016E0000C101F30F700F70B732B762BF008031943
:1016F0007B2B0C147C2B0C101F30F700F70B7E2B70
:10170000812BF1080319862B0C14872B0C101F302A
:10171000F700F70B892B8C2BF2080319912B0C1473
:10172000922B0C101F30F700F70B942B972BF3081C
:1017300003199C2B0C149D2B0C101F30F700F70B7A
:101740009F2BA22BF4080319A72B0C14A82B0C1009
:101750001F30F700F70BAA2BAD2BF5080319B22B9E
:101760000C14B32B0C101F30F700F70BB52BB82B54
:10177000F6080319BD2B0C14BE2B0C101F30F700FC
:10178000F70BC02BC32BFB080319C82B0C14C92B58
:101790000C101F30F700F70BCB2BCE2B0C141F3087
:1017A000F700F70BD12BD42B5A2E8C1FF02B2100D6
:1017B000AA08031DE62BAB08031DE62BAC08031D8E
:1017C000E62BAD08031DE62B2000F02BFF30AA0707
:1017D000031CAB07031CAC07031CAD072000D52B73
:1017E0001F30F700F70BF22BF52B0F30F700F70B3C
:1017F000F72BFA2B8C1FFE2BFC17FF2BFC131F3033
:10180000F700F70B012C042C8C1F082C7C17092CDB
:101810007C131F30F700F70B0B2C0E2C8C1F122C97
:10182000FC16132CFC121F30F700F70B152C182C8C
:101830008C1F1C2C7C161D2C7C121F30F700F70B04
:101840001F2C222C8C1F262CFC15272CFC111F3042
:10185000F700F70B292C2C2C8C1F302C7C15312CED
:101860007C111F30F700F70B332C362C8C1F3A2CD1
:10187000FC143B2CFC101F30F700F70B3D2C402CC8
:101880008C1F442C7C14452C7C101F30F700F70B68
:10189000472C4A2C8C1F512CFE080319512CFE0397
:1018A0004A2C1F30F700F70B532C562C0F30F70043
:1018B000F70B582C5B2C8C1F5F2CFD17602CFD1335
:1018C0001F30F700F70B622C652C8C1F692C7D17DD
:1018D0006A2C7D131F30F700F70B6C2C6F2C8C1FBC
:1018E000732CFD16742CFD121F30F700F70B762CAD
:1018F000792C8C1F7D2C7D167E2C7D121F30F700DD
:10190000F70B802C832C8C1F872CFD15882CFD1148
:101910001F30F700F70B8A2C8D2C8C1F912C7D1516
:10192000922C7D111F30F700F70B942C972C8C1FF5
:101930009B2CFD149C2CFD101F30F700F70B9E2CE8
:10194000A12C8C1FA52C7D14A62C7D101F30F70018
:10195000F70BA82CAB2C0F30F700F70BAD2CB02CED
:1019600021008C131F30F700F70BB42CB72CF008B4
:101970000319BC2C8C17BD2C8C131F30F700F70BF0
:10198000BF2CC22CF1080319C72C8C17C82C8C1340
:101990001F30F700F70BCA2CCD2CF2080319D22CFC
:1019A0008C17D32C8C131F30F700F70BD52CD82CA9
:1019B000F3080319DD2C8C17DE2C8C131F30F70075
:1019C000F70BE02CE32CF4080319E82C8C17E92C16
:1019D0008C131F30F700F70BEB2CEE2CF5080319D6
:1019E000F32C8C17F42C8C131F30F700F70BF62C0C
:1019F000F92CF6080319FE2C8C17FF2C8C131F30C2
:101A0000F700F70B012D042DFB080319092D8C1786
:101A10000A2D8C131F30F700F70B0C2D0F2D8C1790
:101A20001F30F700F70B122D152D5A2E0C1F312DDC
:101A30002100AA08031D272DAB08031D272DAC0884
:101A4000031D272DAD08031D272D2000312DFF304C
:101A5000AA07031CAB07031CAC07031CAD0720003F
:101A6000162D1F30F700F70B332D362D0F30F700F2
:101A7000F70B382D3B2D0C1F3F2DFC17402DFC1371
:101A80001F30F700F70B422D452D0C1F492D7C17F9
:101A90004A2D7C131F30F700F70B4C2D4F2D0C1FD8
:101AA000532DFC16542DFC121F30F700F70B562D4A
:101AB000592D0C1F5D2D7C165E2D7C121F30F700FA
:101AC000F70B602D632D0C1F672DFC15682DFC1185
:101AD0001F30F700F70B6A2D6D2D0C1F712D7C1533
:101AE000722D7C111F30F700F70B742D772D0C1F12
:101AF0007B2DFC147C2DFC101F30F700F70B7E2D86
:101B0000812D0C1F852D7C14862D7C101F30F70035
:101B1000F70B882D8B2D0C1F922DFE080319922D8B
:101B2000FE038B2D1F30F700F70B942D972D0F30F0
:101B3000F700F70B992D9C2D0C1FA02DFD17A12D43
:101B4000FD131F30F700F70BA32DA62D0C1FAA2D98
:101B50007D17AB2D7D131F30F700F70BAD2DB02D8A
:101B60000C1FB42DFD16B52DFD121F30F700F70B1D
:101B7000B72DBA2D0C1FBE2D7D16BF2D7D121F3027
:101B8000F700F70BC12DC42D0C1FC82DFD15C92D55
:101B9000FD111F30F700F70BCB2DCE2D0C1FD22DD2
:101BA0007D15D32D7D111F30F700F70BD52DD82DC6
:101BB0000C1FDC2DFD14DD2DFD101F30F700F70B81
:101BC000DF2DE22D0C1FE62D7D14E72D7D101F303B
:101BD000F700F70BE92DEC2D0F30F700F70BEE2D8A
:101BE000F12D21000C131F30F700F70BF52DF82D08
:101BF000F0080319FD2D0C17FE2D0C131F30F700F4
:101C0000F70B002E032EF1080319082E0C17092ECE
:101C10000C131F30F700F70B0B2E0E2EF2080319D2
:101C2000132E0C17142E0C131F30F700F70B162E63
:101C3000192EF30803191E2E0C171F2E0C131F301C
:101C4000F700F70B212E242EF4080319292E0C1768
:101C50002A2E0C131F30F700F70B2C2E2F2EF50811
:101C60000319342E0C17352E0C131F30F700F70B09
:101C7000372E3A2EF60803193F2E0C17402E0C1360
:101C80001F30F700F70B422E452EFB0803194A2E92
:101C90000C174B2E0C131F30F700F70B4D2E502E48
:101CA0000C171F30F700F70B532E562E5A2E20001C
:101CB00021005A2E22000C16FE0803196D2E210059
:101CC000AA08031DAA2EAB08031DAA2EAC08031DEB
:101CD000AA2EAD08031DAA2E22002100BE0102304B
:101CE000BF008031200086258831FF30230091001D
:101CF00001309200803120004F2688312100BE0142
:101D00000330BF0080312000862588312100AA08D9
:101D1000031D9E2EAB08031D9E2EAC08031D9E2E98
:101D2000AD08031D9E2E0A30230091000230920060
:101D3000803120004F268831A72E21001530230046
:101D4000910002309200803120004F26883121001E
:101D5000BA011B2FFC08031DB62EFD08031DB62E6D
:101D6000AF012F08AE000130BA001B2FBA080319CB
:101D70001B2F2F08CB001430CC00803120008F2582
:101D8000883121002E0878070A3E84002030850023
:101D90000318850A7C0880002F08CB001430CC0083
:101DA000803120008F25883178082100BD00013066
:101DB0002E073D070A3E8400203085000318850A5F
:101DC0007D0880000230AE072E08143C031DEE2E65
:101DD000AE01AF0A2F08043C0319AF013008BE0062
:101DE0003108BF008031200086258831210031086C
:101DF000CB001430CC00803120008F2588312100A9
:101E0000300878070A3E8400203085000318850AD0
:101E10000008BD00C50080312000B62588312100B2
:101E2000B00A3008143C031D1B2FB001B10A310861
:101E3000043C0319B10120000D1A502F21003C0B66
:101E4000222F242F2000502F2000A50A0330A505A3
:101E500014302300910020002508230093009513DF
:101E600015150B08F7008B1355309600AA30960015
:101E700095149518392F151177088B042000250823
:101E80002100BD00803120008C2788316430210082
:101E9000BD0080312000542288312100BC01200087
:101EA0000D1E562F01302100BC0020000529210005
:101EB00088312000EE2F850184011F308305F43026
:101EC000210099002000A801A9013230FE00210064
:101ED000AE01AF01B001B10123008C018D012200E0
:101EE0009201910194019301F03021009900023098
:101EF000B600FA30BD008031200054228831210024
:101F0000B60B792F80312000692A88316430210096
:101F1000BD0080312000542288318031892A8831E7
:101F2000F8080319962F8031DE2A88318031DE2BA4
:101F300088318D1E9D2FA0019F2F0130A000803180
:101F4000A02C88318031EF2488312100BE01BF01EF
:101F500080312000862588313D30230091000230F9
:101F60009200803120004F2688312100BE010230CE
:101F7000BF00803120008625883146302300910043
:101F800002309200803120004F2688312100BE01AE
:101F90000630BF0080312000862588314D30230077
:101FA000910002309200803120004F2688310430A9
:101FB0002100B600FA30BD00803120005422883163
:101FC0002100B60BDA2F20000D1AEA2F8031EF2402
:0E1FD000883100288031EF248831EB2863002F
:020000040001F9
:04000E008439FF1E14
:00000001FF
